:100D00002A4D4553534147453A20615F7374203D56
:100D10002025750D0A002A4D4553534147453A2079
:100D200061283029203D2025750D0A002A5741529F
:100D30004E494E473A20416363656C657261746940
:100D40006F6E206F7574206F662072616E67653AF2
:100D500020615F73743D25752C2061303D25750D34
:100D60000A002A4D4553534147453A2070283029FF
:100D7000203D2025750D0A002A5741524E494E4705
:100D80003A205072657373757265202575206F75F2
:100D900074206F662072616E6765205B25752C2557
:100DA000755D0D0A002A5741524E494E473A20427E
:100DB0007265616B77697265206E6F7420636F6E08
:100DC0006E656374656420286E6F20666C69676861
:100DD00074290D0A002020202020200D0A002A5608
:100DE000455253494F4E3A20522D444153205632DA
:100DF0002E312E310D0A002A4D4553534147453AB5
:100E00002053656C667465737420706173736564D8
:100E10000D0A002A5741524E494E473A2053656CFD
:100E20006674657374206661696C65640D0A002AD6
:080E300052454144590D0A002E
:07206F00EF60031F80FA225D
:101EDA00A2099293E4F559F55A7F7812206F055AB0
:0F1EEA00E55A70020559E55A6464455970EB22B8
:100E3800D209121EDA7F06121DDC907CB2EEF0A3F6
:100E4800EFF0C209121EDA7BFF7A0D7900907CB2AE
:100E5800E0FFA3E0907C8CCFF0A3EFF01200C97FF5
:100E680006121DDC907CB4EEF0A3EFF07BFF7A0D48
:100E78007916907C8CEEF0A3EFF01200C9907CB448
:100E8800E0FEA3E0FF907CB2E0FCA3E0FDC39FFF7F
:100E9800EC9EFEC3EF942DEE6480948050297BFF76
:100EA8007A0D792C907C8CECF0A3EDF0907CB4E07A
:100EB800FFA3E0907C8ECFF0A3EFF01200C97F066D
:100EC80012000EC218C3227F07121DDC907CB2EEFE
:100ED800F0A3EFF07BFF7A0D7962907C8CEEF0A3A3
:100EE800EFF01200C9907CB2E0FEA3E0FFC3947D4E
:100EF800EE64809482400BD3EF94DBEE648094839D
:100F080040287BFF7A0D7978907C8CEEF0A3EFF087
:100F1800A37402F0A3747DF0A37403F0A374DBF050
:100F28001200C97F0512000EC32230131DA294308F
:100F38001401B34015755D047BFF7A0D79A5120085
:100F4800C97F0412000EC213C3227F0112000ED300
:010F58002276
:1018E200D2AF121F4C121F1712208012205D12203D
:1018F200767BFF7A0D79D51200C97BFF7A0D79DEEE
:101902001200C9120E38500B7BFF7A0D79F71200C4
:10191200C980097BFF7A0E79131200C912187C90D4
:101922007CDEE0FF121C1C121E98121B04907CDF4E
:10193200E0FEA3E0FF121B987BFF7A0E792F1200C4
:05194200C9121F66221E
:03000B00021A08CE
:101A0800C0E0C0F0C083C082C0D075D008E549F5F9
:101A18008CE54AF58AD54E09907CD8E0F54E121E21
:101A2800B9D54D17907CD8E0F54D054CE54C7002C2
:101A3800054BE54C454B7003755D05E55D64046039
:101A48000912117C121734121D59D0D0D082D083BC
:051A5800D0F0D0E032E7
:101B9800E4FCFDFB7AC079A8F81204687BE07A2E91
:101BA80079007800121B54C3E49FF54AE49EF54976
:101BB800907CD8E0F54EF54DE4F54BF54CE58954AD
:101BC800F04401F589758CFF758AFFC2B9D2A9D294
:021BD8008C225D
:0C202F00907CD8E0F54DE4F54BF54C2218
:101B0400E5C520E3FB75C50775C50FE5C530E4FBE6
:101B1400AFC6EF75F004A4FFAEF0E5C5C4131354CB
:101B2400037C002FF52DEC3EF52CE4F52BE52B255D
:101B3400E0245FF8A62C08A62DE52D2528F528E538
:101B44002C3527F527052BE52BB40AE1E4F52A22E9
:10117C00C0D075D008301B0302127DE5C520E3FBFF
:10118C00E4F5C575C508F533753401E533640870AD
:10119C000302125FE5C530E4FB85C62985C52EE543
:1011AC00336407600EE5C520E3FBE53304F5C54465
:1011BC0008F5C5907CD7E055347003021254AF2962
:1011CC00121CC3AF2E121CC3E533B4061BE52975E4
:1011DC00F004A4FFAEF0E52EC4131354037C002FCF
:1011EC00F532EC3EF5318060E5336407705AE52A40
:1011FC0025E02460F8C3E52896F528E5271896F530
:10120C0027E52975F004A4FFAEF0E52EC4131354A2
:10121C00037C002FF536EC3EF535E52A25E0245FFE
:10122C00F8A63508A636E5362528F528E535352700
:10123C00F527FEAF287D0A1203E78E258F26052A97
:10124C00E52AB40A03E4F52A0533E53425E0F53440
:10125C0002119730171BE4A2C492E4A2C592E5A236
:10126C009692E6A29792E7255DC4F52FAF2F121C3C
:04127C00C3D0D022E9
:1017A500C0D075D008301765907CDEE0FD7C0090D8
:1017B5007CE5E0FB24FFFFE434FFFE1203D3EF24B6
:1017C50001FFE43EFEC3E51F9FF51FE51E9EF51EC6
:1017D5008B30E5306021E51EF583E51FF582E0C419
:1017E50054F0255DC4F0907CDEE0251FF51FE4353F
:1017F5001EF51E153080DB907CDEE024FFFFE4340F
:10180500FFFEC3E51F9FF51FE51E9EF51ED0D022E6
:1020120053544F52452069732066756C6C0D0A004B
:0D202200E4F556F557F558C21B121C552267
:10173400C0D075D008E55D6065201B62121FBA40F9
:101744005D907CDEE025E0907CB1F0907CB1E060BF
:101754004D20194A121CF78F55121D860557E5575F
:10176400700205567004E5566480702AF556F557E4
:101774000558E558B40C127BFF7A2079121200C97F
:101784007F0312000ED21B8015121FA7E55820E01C
:1017940005121C558008907CB1E014F080ADD0D0C7
:0117A4002222
:101BDA00464C494748545F4C61756E63680D0A006C
:101BEA00464C494748545F456A656374506172615F
:101BFA006368757465310D0A00464C494748545F5D
:101C0A00456A656374506172616368757465320D03
:021C1A000A00BE
:101E9800E4907C86F0A3F0907C041204EC0000002F
:101EA8000074FF907C00F0A3F0E4907C88F0F55D6E
:011EB8002207
:101EF900C0D075D0087BFF7A1B79DA1200C9755DED
:0E1F090001C2901220227F0212000ED0D022C0
:101E2C00C0D075D0087BFF7A1B79EA1200C9C29129
:101E3C00E54C2401907C03F0E4354B907C02F0756A
:051E4C005D02D0D02270
:101E5100C0D075D0087BFF7A1C79031200C9C292E9
:101E6100E54C2401907C03F0E4354B907C02F07545
:051E71005D03D0D0224A
:10160700C0D075D00830131EA294301401B3401611
:10161700C21D12202F907CD5E0FEA3E0FF121D2BE8
:10162700121EF90216B42018030216B4907CD3E0F8
:10163700FEA3E0FFC3E5469FFFE5459EFED3E532E7
:101647009FE5319E4016D21D907C041204EC0000E9
:101657000000E4907C86F012202F8051C21D907C00
:1016670004E0F8A3E0F9A3E0FAA3E0FBC3E53295B1
:1016770046FFE5319545FE3395E0FDFCEB2FFFEA8C
:101687003EFEE93DFDE83CFC907C041204E0907CC2
:10169700E5E0FF907C86E004F06F7011907CD9E064
:1016A700FEA3E0FF121D2B121EF91217A5D0D022A0
:1016B700C0D075D008907C04E0F8A3E0F9A3E0FA65
:1016C700A3E0FBC3E5329546FFE5319545FE33952B
:1016D700E0FDFCEB2FFFEA3EFEE93DFDE83CFC9018
:1016E7007C041204E03016307F007E007D007C0011
:1016F700907C04E0F8A3E0F9A3E0FAA3E0FBD3129F
:1017070004B74014907CD2E0FFD3E54C9FE54B949F
:10171700004005121E2C801230150F907CE3E06507
:0D1727004C7002E54B7003121E2CD0D02236
:10194700C0D075D008907C02E0FEA3E0654C700320
:10195700E54B6E7002D291301634907CDCE0FEA32A
:10196700E0FFC3E5489FFFE5479EFEC3E5269FE5E9
:10197700259E5007E4907C87F08013907CE6E0FF7B
:10198700907C87E004F06F7005121E5180123015AD
:101997000F907CE4E0654C7002E54B7003121E511A
:0319A700D0D0227B
:101F3200C0D075D008907C02E0FEA3E0654C70032F
:0A1F4200E54B6E7002D292D0D0225F
:101D5900C0D075D008E55D7005121607801CE55DD9
:101D6900B401051216B78012E55DB40205121947D0
:0D1D79008008E55DB40303121F32D0D022B4
:101C1C00CBEFCBEBFD7C007E507F001203E7CDEBCE
:101C2C00CD7C001203D38E1A8F1B74002FF582EE1D
:101C3C00342CAF82F5188F197E2C7F008E1C8F1DD3
:091C4C008E1E8F1FD219C21A224C
:101CC300C219051FE51FAC1E7002051E14F5828C98
:101CD30083EFF0E51F65197004E51E65187006753E
:101CE3001E2C751F00E51F651D7004E51E651C7025
:041CF30002D21A22DD
:101CF700C21A051DE51DAE1C7002051C14F5828E67
:101D070083E0FFE51D65197004E51C65187006750D
:101D17001C2C751D00E51F651D7004E51E651C70F4
:041D270002D21922A9
:101D2B00C3E51F9FF51DE51E9EF51CC3E51D940025
:101D3B00E51C942C400BD3E51D9519E51C9518401B
:0E1D4B000CE51B251DF51DE51A351CF51C22A7
:1009120063202562752025627520257520257520A6
:1009220025627520256275202563202562752025A4
:10093200632025632025630D0A0074696D6500201C
:1009420020616463257500206469676974616C00C5
:100952000D0A002D2D2D2D2D2D2D2D2D2D2D2D2D35
:100962002D2D2D2D2D2D2D2D2D2D2D2D2D2D2D2DB5
:100972002D2D2D2D2D2D2D2D2D2D2D2D2D2D2D2DA5
:100982002D2D2D2D2D2D2D2D2D2D2D2D2D2D2D2D95
:100992002D2D2D2D2D2D2D2D2D2D2D2D2D2D2D2D85
:1009A2002D0D0A002533753A002025303262580099
:1009B2003A2530326258002020202533750020303D
:1009C20078253032627800436865636B73756D3DDC
:1009D2003078253034580D0A002A4D45535341478B
:1009E200453A205265616420636F6E6669673A20FA
:1009F20020633F0D0A002A4D4553534147453A2093
:100A0200416C74657220636F6E6669673A20632079
:100A120066722061752061742070642074312074C4
:100A220032206469206277206773207370207470AB
:100A32000D0A002A4D4553534147453A2053746FDE
:100A4200726520636F6E6669673A2063210D0A0042
:100A52002A4D4553534147453A20446F776E6C6F98
:100A620061643A20202020206420740D0A002A4D5F
:100A72004553534147453A2044756D703A20202032
:100A82002020202020207520740D0A002A4D455375
:100A9200534147453A2044756D70206865783A2085
:100AA20020202020757820740D0A002A4D455353CA
:100AB2004147453A2048656C703A2020202020208A
:100AC200202020680D0A002A4D4553534147453ADC
:100AD2002052657365743A20202020202020207245
:100AE200657365740D0A002A4D4553534147453AD3
:100AF2002056657273696F6E3A202020202020767E
:100B02000D0A002A56455253494F4E3A20522D445F
:100B120041532056322E312E310D0A007265736513
:100B220074007066007064002A4552524F523A2097
:100B3200556E6B6E6F776E20636F6D6D616E640DB7
:020B42000A00A7
:06207600E4F55EC21C222D
:100B4400301313301408907CCC7401F0800D907C29
:100B5400CC7402F08005E4907CCCF0907CE8E064F6
:100B64003F6003020BF27BFF7A097912907CD8E094
:100B7400907C8CF0907CD7E0907C8DF0907CD3E0DE
:100B8400FFA3E0907C8ECFF0A3EFF0907CDCE0FF3D
:100B9400A3E0907C90CFF0A3EFF0907CE3E0907C16
:100BA40092F0907CE4E0907C93F03017047F3180E5
:100BB400027F30907C94EFF0907CCCE0907C95F0B8
:100BC4003018047F3180027F30907C96EFF030162D
:100BD400047F3180027F30907C97EFF03015047FE2
:100BE4003180027F30907C98EFF01200C922907C13
:100BF400E8E0B4210412128022907CC97401F0A3AD
:100C0400747CF0A374E8F0907CC9E0FBA3E0FAA341
:100C1400E0F91203BAFF121F7E500C907CCAE475EF
:100C2400F00112043C80E0E4907CC8F0907CC9E0C0
:100C3400FBA3E0FAA3E0F912146D907CC8E025E070
:100C440024B2F582E4347CF583EEF0A3EFF0907CDB
:100C5400C9E0FBA3E475F001120452A9F0FA1203EF
:100C6400BAFF121F7E50E7907CC8E004F0E0B40B9A
:100C7400BB907CB3E0907CD8F0907CB5E0907CD7BE
:100C8400F0907CB6E0FFA3E0907CD3CFF0A3EFF02C
:100C9400907CB8E0FFA3E0907CDCCFF0A3EFF09071
:100CA4007CBBE0907CE3F0907CBDE0907CE4F09031
:100CB4007CBEE0FEA3E0FFEE4F24FF9217A3E0FE0C
:100CC400A3E0FFEE4F24FF9213EF64014E7003D3B1
:100CD4008001C39214907CC2E0FEA3E0FFEE4F2497
:100CE400FF9218A3E0FEA3E0FFEE4F24FF9216A3A9
:0C0CF400E0FEA3E0FFEE4F24FF9215226B
:101382007B017A7C79E812106EC8ECC8C9EDC9CA33
:10139200EECACBEFCB907CE1E0FEA3E0FFE4FCFDE4
:1013A200120468C8ECC8C9EDC9CAEECACBEFCB902B
:1013B2007CD5E0FEA3E0FFE4FCFDEB2FFFEA3EFE5E
:1013C200ED39FDEC38FC907CB41204E0907CB4E082
:1013D200FCA3E0FDA3E0FEA3E0FF780F1204CD8F93
:1013E20058907CB4E0FCA3E0FDA3E0FEA3E0FFEE96
:1013F200547FFEE48E568F57121FA7E4907CB8F0FC
:10140200A3F0907CB2F0A3F0907CE1E0FEA3E0FFB9
:10141200907CB2E06E7003A3E06F603E12203BEF5F
:10142200FD907CB9E02DF0907CB8E03400F0120021
:10143200030557E557700205567004E5566480703F
:1014420009F556F5570558121FA7907CB3E004F032
:101452007006907CB2E004F080AE907CB8E0FF129F
:0B1462000003907CB9E0FF12000322A1
:101E050012203B907CBEEFF00557E5577002055652
:101E15007004E55664807009F556F5570558121F8C
:071E2500A7907CBEE0FF2244
:10067E00907CE8E0B47803D38001C3920930094E30
:10068E007B017A7C79E912106EC8ECC8C9EDC9CA33
:10069E00EECACBEFCB907CE1E0FEA3E0FFE4FCFDE5
:1006AE00120468C8ECC8C9EDC9CAEECACBEFCB902C
:1006BE007CD5E0FEA3E0FFE4FCFDEB2FFFEA3EFE5F
:1006CE00ED39FDEC38FC907CB61204E0804C7B01D9
:1006DE007A7C79E812106EC8ECC8C9EDC9CAEECAA8
:1006EE00CBEFCB907CE1E0FEA3E0FFE4FCFD120437
:1006FE0068C8ECC8C9EDC9CAEECACBEFCB907CD5A1
:10070E00E0FEA3E0FFE4FCFDEB2FFFEA3EFEED3939
:10071E00FDEC38FC907CB61204E0907CB6E0FCA3B5
:10072E00E0FDA3E0FEA3E0FF780F1204CD8F5890FA
:10073E007CB6E0FCA3E0FDA3E0FEA3E0FFEE547F59
:10074E00FEE48E568F57121FA77BFF7A09793C1253
:10075E0000C9907CB57401F0E4907CB2F0A3F090E7
:10076E007CB5E0FF6037907CD7E05F60187BFF7A46
:10077E00097941907CB2E0FFA3E0907C8CCFF0A38E
:10078E00EFF01200C9907CB5E0FF25E0F0907CB34D
:10079E00E004F07006907CB2E004F080C2301709DD
:1007AE007BFF7A0979491200C97BFF7A09795212C7
:1007BE0000C97BFF7A0979551200C9E4907CBCF020
:1007CE00A3F0907CB2F0A3F0907CD8E0FF907CB2C6
:1007DE00E0FCA3E0FDEF6D7001EC70030208F97B05
:1007EE00FF7A0979A6907C8CECF0A3EDF01200C98B
:1007FE00907CB57401F0907CB5E0FF70030208B6F2
:10080E00907CD7E05F70030208AB121E05907CB49B
:10081E00EFF030090E7BFF7A0979ABE0907C8CF01B
:10082E001200C9907CB4E0FF7E00907CBDE02FF0FA
:10083E00907CBCE03EF0EF75F004A4907CBBF0E53C
:10084E00F0907CBAF0121E05907CB4EFF030090ED9
:10085E007BFF7A0979B2E0907C8CF01200C9907C13
:10086E00B4E0FFFD907CBDE02DF0907CBCE0340048
:10087E00F0EFC413135403FF907CBBE02FF0907C79
:10088E00BAE03400F02009157BFF7A0979B9E0FF50
:10089E00A3E0907C8CCFF0A3EFF01200C9907CB552
:1008AE00E0FF25E0F0020804301726121E05907CAA
:1008BE00B4EFF0E0FFFD907CBDE02DF0907CBCE04D
:1008CE003400F07BFF7A0979C0907C8CEFF0120037
:1008DE00C97BFF7A0979521200C9907CB3E004F00B
:1008EE007006907CB2E004F00207D67BFF7A09799D
:1008FE00C9907CBCE0FFA3E0907C8CCFF0A3EFF01E
:04090E001200C922E8
:101AB2007BFF7A0979DB1200C97BFF7A0979F81278
:101AC20000C97BFF7A0A79351200C97BFF7A0A794D
:101AD200521200C97BFF7A0A79701200C97BFF7A21
:101AE2000A798E1200C97BFF7A0A79AD1200C97B8E
:101AF200FF7A0A79C91200C97BFF7A0A79E91200D2
:021B0200C922F6
:04207C00121E762298
:0A2053007BFF7A0B79051200C92209
:10154500907CE7E0B46304120B4422907CE7E0B49E
:10155500640412138222907CE7E0B46804121AB284
:1015650022907CB574FFF0A3740BF0A3741EF0A356
:10157500E4F0A37405F07B017A7C79E7121815EF86
:10158500700412207C22907CB574FFF0A3740BF0DC
:10159500A37424F0A3E4F0A37402F07B017A7C79B0
:1015A500E7121815EF700D7B017A7C79EB12146D3B
:1015B500121FDF22907CB574FFF0A3740BF0A374A7
:1015C50027F0A3E4F0A37402F07B017A7C79E7129B
:1015D5001815EF700D7B017A7C79EB12146D121FD3
:1015E500F022907CE7E0B4750412067E22907CE739
:1015F500E0B47604122053227BFF7A0B792A12007D
:02160500C922F8
:101F6600101C0280FB755D047F0112000E7F1E129D
:081F76001FCD12154580E92280
:10002600C0D0EF20E72CEF640A6027EF640D601163
:1000360074E7255EF582E4347CF583EFF0055E8097
:100046001174E7255EF582E4347CF583E4F0D21C76
:05005600F55ED0D02290
:101A5D002A4D4553534147453A2053746F72696E71
:101A6D006720706172616D657465727320696E2097
:101A7D00464C4153480D0A002A4D455353414745A5
:101A8D003A2046696E69736865642073746F726974
:101A9D006E670D0A00000001C001C802000C003283
:051AAD000001193C03DB
:0A205D00755B1A755CA2120F592280
:100F5900901AA2E49324FF9213A3E49324FF92141A
:100F6900A3E49324FF9218A3E493907CD7F0901AFA
:100F7900A6E49324FF9217E4907CDEF07F80EF6073
:100F890014907CD7E05F6007907CDEE02402F0EFEC
:100F9900C313FF80E9301706907CDEE004F0901A55
:100FA900A7E493907CD8F0901AA8E493907CDBF0A6
:100FB900901AA9E493FF740193907CD3CFF0A3EF27
:100FC900F0901AABE493FF740193907CDCCFF0A30B
:100FD900EFF0907CD8E0FBFD7C007E037FE81203F4
:100FE900E7907CDFEEF0A3EFF0907CDEE0FA8BF087
:100FF900A4FF907CE1E5F0F0A3EFF0EB1313543F6D
:10100900907CE5F0FBA3F0901AADE49324FF9216CF
:10101900A3E49324FF9215A3E493907CE3F0901A40
:10102900B0E493907CE4F0901AB1E493907CD2F010
:10103900907CDBE0FF7E00907CE1E0FCA3E0FD1208
:1010490003D3907CD5EEF0A3EFF0EBFF7E00EAFD31
:101059007C001203D3E02F907CDAF0907CD5E03E3F
:05106900907CD9F0228B
:10128000A213E433855C82855B83F0A214E433A36C
:10129000F0A218E433855C82855B83A3A3F0907C85
:1012A000D7E0855C82855B83A3A3A3F0A217E43318
:1012B000FFE55C2404F582E4355BF583EFF0907C78
:1012C000D8E0FFE55C2405F582E4355BF583EFF0BB
:1012D000907CDBE0FFE55C2406F582E4355BF5837A
:1012E000EFF0907CD3E0FEA3E0FFE55C2407F582FD
:1012F000E4355BF583EEF0A3EFF0907CDCE0FEA339
:10130000E0FFE55C2409F582E4355BF583EEF0A3AC
:10131000EFF0A216E433FFE55C240BF582E4355BC5
:10132000F583EFF0A215E433FFE55C240CF582E4CD
:10133000355BF583EFF0907CE3E0FFE55C240DF591
:1013400082E4355BF583EFF0907CE4E0FFE55C241C
:101350000EF582E4355BF583EFF0907CD2E0FFE59B
:101360005C240FF582E4355BF583EFF07BFF7A1A9E
:10137000795D1200C9121C8E7BFF7A1A79851200E2
:02138000C92280
:10187C00E5C520E3FB75C50675C50EE5C530E4FB73
:10188C00AFC6EF75F004A4FFE5C5C4131354037C75
:10189C00002FFFEC35F0CF2401F542E43FF541F584
:1018AC0045854246E5C520E3FB75C50775C50FE5C3
:1018BC00C530E4FBAFC6EF75F004A4FFAEF0E5C590
:1018CC00C4131354037C002FF544EC3EF543F54749
:0618DC00854448D21D22E4
:101EB900301D1D854145854246E5322401F542E440
:101EC9003531F54185434785444885254385264471
:011ED90022E6
:101F4C00C21E43878075985AE589540F4420F58941
:0A1F5C00758DFFD28ED2BCD2AC22EC
:03002300021DB308
:101DB300C0E0C0F0C083C082C0D075D01030980797
:101DC300AF99C298120026309904C299D21ED0D07E
:091DD300D082D083D0F0D0E032C0
:080003008F99301EFDC21E2280
:082067008F99301EFDC21E22FC
:101DDC00E5C520E3FB8FC5EF4408F5C5E5C530E448
:101DEC00FBAFC6EF75F004A4FFAEF0E5C5C413134A
:091DFC005403FDE5F0EF4DFF2258
:101E7600E4F5A8F5E8F5B8F5F875580FE558A2E0C9
:101E860092B5A2E192B3A2E292B4A2E392B202FFA9
:021E9600FE222A
:101FA700E558A2E092B5A2E192B3A2E292B4A2E30D
:031FB70092B222C1
:0C203B00E5564480855782F583E0FF22C3
:101D860090D3557499F090ACAA7466F090D35574BC
:101D960090F0E555F5F0E556D2E7F583E557F5827F
:0D1DA600E5F0F0E0A2E730F701B340F722CE
:101C5500E558A2E092B5A2E192B3A2E292B4A2E362
:101C650092B290D3557499F090ACAA7466F090D363
:101C7500557480F090D3557499F090ACAA7466F0C1
:091C85009080007414F0D21F22BB
:101FBA00301F0D908000E020E703D38001C3921FF9
:031FCA00A21F2231
:101C8E0075580C121C55121FBA40FB75580D121FB9
:101C9E00A7E4F556F557855782855683E0F555121C
:101CAE001D860557E55770020556E5577004E55633
:051CBE00648070E222C9
:03208000C21F225A
:101F930050574D503D2562750A00447574793D25AF
:041FA30062750A0059
:03005B000219AADD
:1019AA00C0E0C0D0C2CC742D25C9F5C930204A1573
:1019BA004FE54F7044E554700F8551FCC2C0F55095
:1019CA00755401754F028031E554B4011C75FCFF52
:1019DA00D2C00550E55065527007F55485534F80C3
:1019EA0018755402754F028010E554B4020B8551E4
:0E19FA00FCC2C0755401754F02D0D0D0E0324F
:101F170075FCFFD2C075FE0B75518075EA0DC2FCCA
:0B1F2700D2EC75530A7F0112000E225D
:10000E00C22075FCFFD2C08F52E4F55485534FEFDA
:05001E006002D2202267
:101FCD00C22075FCFFD2C08F53E4F55485534FD218
:021FDD002022C0
:101FDF008FFE7BFF7A1F7993907C8CEFF01200C9F4
:011FEF0022CF
:101FF0008F517BFF7A1F799D907C8CEFF01200C986
:0120000022BD
:0300000002204794
:0C204700787FE4F6D8FD7581720218E283
:1003BA00BB010689828A83E0225002E722BBFE0241
:0903CA00E32289828A83E4932274
:1003D300EFF88DF0A4FFEDC5F0CEA42EFEEC88F06F
:0403E300A42EFE2224
:1003E700BC000BBE0029EF8DF084FFADF022E4CCFA
:1003F700F875F008EF2FFFEE33FEEC33FCEE9DECC3
:10040700984005FCEE9DFE0FD5F0E9E4CEFD22ED08
:10041700F8F5F0EE8420D21CFEADF075F008EF2F52
:10042700FFED33FD4007985006D5F0F222C398FD43
:050437000FD5F0EA22E0
:10043C00C5F0F8A3E028F0C5F0F8E582158270024B
:06044C001583E038F022E8
:10045200A3F8E0C5F025F0F0E5821582700215835D
:06046200E0C838F0E822BA
:10046800E88FF0A4CC8BF0A42CFCE98EF0A42CFC33
:100478008AF0EDA42CFCEA8EF0A4CDA8F08BF0A4B1
:100488002DCC3825F0FDE98FF0A42CCD35F0FCEB10
:100498008EF0A4FEA9F0EB8FF0A4CFC5F02ECD39D5
:0F04A800FEE43CFCEAA42DCE35F0FDE43CFC2242
:101B5400C2D5E830E70FB2D5E4C39BFBE49AFAE4BC
:101B640099F9E498F8EC30E717B2D5121B8A1205FC
:101B740098E4C39BFBE49AFAE499F9E498F88003A7
:101B840012059830D50DE4C39FFFE49EFEE49DFD4D
:041B9400E49CFC22AF
:1004B700EB9FF5F0EA9E42F0E99D42F0EC6480C8BC
:0604C70064809845F0225C
:1004CD00E8600FECC313FCED13FDEE13FEEF13FF0D
:0304DD00D8F12231
:0C04E000ECF0A3EDF0A3EEF0A3EFF0228F
:1004EC00A8828583F0D083D08212050312050312F3
:1004FC000503120503E473E493A3C583C5F0C58318
:10050C00C8C582C8F0A3C583C5F0C583C8C582C859
:01051C0022BC
:10005E00E53C248CF582E4347CF583E0053C22906B
:10006E007C89301103907C8CE475F0011206380205
:10007E0003BA200AE97F2ED20A8018EF540F24907B
:10008E00D43440D4FF300E0BEF24BFB41A0050030B
:10009E002461FFE53D6002153D0540E54070020517
:1000AE003F30110E907C89E475F001120638EF0294
:1000BE00054A0220677403D2118003E4C211F53C95
:1000CE00907C8912064FE4F53DF53FF540E53D6025
:1000DE00077F201200A180F5F53EC20BC20AC20CAA
:1000EE00C20DC20FC210C21212006DFF700D301180
:1000FE00057F001200B2AF40AE3F22B42561C2D5DB
:10010E00C20E12006DFF24D0B40A00501C75F00A06
:10011E0020D50DC53DA4253DF53D7002D20D80E0E4
:10012E00C53EA4253EF53E80D724CFB41A00EF502D
:10013E0004C2E5D20E0202ACD20B80C4D20A80BE3B
:10014E00D20C80BAD2D580B8D20F80B27F201200E6
:10015E00A1200C077401B53D0040F112005EFF12A4
:10016E0000A10200DBD212D210809312005EFB12AD
:10017E00005EFA12005EF94A4B700679787A037BBC
:10018E00FF200C33E53D602FAF3EBF00011F7E0008
:10019E008E8275830012051D60050EEE6F70F1C222
:1001AE00D5EBC0E0EAC0E0E9C0E0EE1202F0D0E02C
:1001BE00F9D0E0FAD0E0FB1203BAFF60A5EBC0E085
:1001CE00EAC0E0E9C0E01200A1D0E02401F9D0E0DD
:1001DE003400FAD0E0FBE53E60DDD53EDA80837B6D
:1001EE00FF7A0279ECD20C8098791080027908C2DD
:1001FE0010C2128008D2D5790A8004790AC2D5E4D9
:10020E00FAFDFEFF12005EFC7B08200B1312005E4F
:10021E00FD7B10300A0A12005EFE12005EFF7B208C
:10022E00EC3382D592D55013C3E4300A069FFFE417
:10023E009EFEE4200B039DFDE49CFCE4CBF8C20B78
:10024E00EC700CCFCECDCCE824F8F870F38017C349
:10025E00EF33FFEE33FEED33FDEC33FCEB33FB9966
:10026E004002FB0FD8E9EB300B05F8D0E0C448B2E2
:10027E000BC0E00AEC4D4E4F78207B0070C2EAC0F6
:10028E00E01202F2D0F0D0E0200B04C4C0E0C4B201
:10029E000BC0F012008AD0F0D5F0EB0200DB120694
:1002AE005801795301F758014A4C01464201FB4F60
:1002BE00020344020349015F4302095501ED460161
:1002CE00ED4501ED47039B50014E2D01522E017558
:1002DE002B01562301732003862A0000016D3F3F38
:1002EE003F00790AA2D5200D14300F09B91002046F
:1002FE0004B9080104A2D5201002500104200C6696
:02030E00920C4F
:10031000B53D005032C0E07F20300D177F30A20C79
:100320007210720F500D120347C20CC210C20F7F21
:1003300030800F300F03E9C0E01200A1300F03D06E
:10034000E0F9D0E0B53DCE300F177F30B9100C1278
:1003500000A17F58300E077F788003B90803120090
:10036000A1300C057F2D0200A17F202012F87F2BE9
:100370002010F322920C80CF286E756C6C29002D12
:1003800050434958D20B12005E300BF8C20B783D37
:1003900030D504D20A783EF602010C12005E240326
:1003A000B405004001E490037F93120092743A1266
:0A03B0000092D20D753D040201F722
:101F7E00EFC394094006EFC3940E4004EFB4200360
:051F8E00D38001C32215
:10181500907CB2EBF0A3EAF0A3E9F0907CB5E0FB95
:10182500A3E0FAA3E0F91203BAFE907CB2E0FBA3B1
:10183500E0FAA3E0F91203BAFD6E702AED600E908E
:101845007CB874FFF5F012043C45F070037F00226C
:10185500907CB3E475F00112043C907CB6E475F01D
:101865000112043C80B5D3EE6480F8ED64809840A5
:07187500037F01227FFF2227
:10106E00907CBEEBF0A3EAF0A3E9F0907CBEE0FB2F
:10107E00A3E0FAA3E0F91203BAFF121F7E500C9000
:10108E007CBFE475F00112043C80E0D20A907CBE75
:10109E00E0FBA3E0FAA3E0F91203BAFF642B6004AD
:1010AE00EFB42D1D907CBEE0FBA3E475F00112049D
:1010BE0052A9F0FA1203BA642D6003D38001C392D1
:1010CE000A907CC11204EC00000000907CBEE0FB94
:1010DE00A3E0FAA3E0F91203BAFF122001506A7FCF
:1010EE000A7E007D007C00907CC1E0F8A3E0F9A3AD
:1010FE00E0FAA3E0FB120468C8ECC8EDC0E0EEC055
:10110E00E0EFC0E0907CBEE0FBA3E0FAA3E0F912B2
:10111E0003BAFF3395E0FEEF24D0FFEE34FFFEE47A
:10112E00FCFDD0E0FBD0E0FAD0E0F9EB2FFFEA3E79
:10113E00FEED39FDEC38FC907CC11204E0907CBFD2
:10114E00E475F00112043C8082300A10907CC1E0FC
:10115E00FCA3E0FDA3E0FEA3E0FF8011907CC1E0C4
:0E116E00FCA3E0FDA3E0FEA3E0FF12062A2290
:10146D00907CCDEBF0A3EAF0A3E9F0907CCDE0FB0E
:10147D00A3E0FAA3E0F91203BAFF121F7E500C90FD
:10148D007CCEE475F00112043C80E0D209907CCD55
:10149D00E0FBA3E0FAA3E0F91203BAFF642B6004AA
:1014AD00EFB42D1D907CCDE0FBA3E475F00112048B
:1014BD0052A9F0FA1203BA642D6003D38001C392CE
:1014CD0009E4907CD0F0A3F0907CCDE0FBA3E0FA92
:1014DD00A3E0F91203BAFF122001503F907CCDE03A
:1014ED00FBA3E0FAA3E0F91203BAFF3395E0FEEF98
:1014FD0024D0FBEE34FFFA907CD0E0FEA3E0FF7C1D
:10150D00007D0A1203D3EF2BF0EE3A907CD0F090D1
:10151D007CCEE475F00112043C80AD30090A907C5C
:10152D00D0E0FEA3E0FF800F907CD0E0FEA3E0FFB3
:08153D00C3E49FFFE49EFE22BF
:10051D00BB010CE58229F582E5833AF583E0225093
:10052D0006E92582F8E622BBFE06E92582F8E222DD
:0D053D00E58229F582E5833AF583E49322F7
:10054A00BB010689828A83F0225002F722BBFE0190
:02055A00F3228A
:10055C0075F008758200EF2FFFEE33FECD33CDCC56
:10056C0033CCC58233C5829BED9AEC99E5829840D9
:10057C000CF582EE9BFEED9AFDEC99FC0FD5F0D6B6
:10058C00E4CEFBE4CDFAE4CCF9A88222B800C1B9E0
:10059C000059BA002DEC8BF084CFCECDFCE5F0CB1E
:1005AC00F97818EF2FFFEE33FEED33FDEC33FCEB57
:1005BC0033FB10D703994004EB99FB0FD8E5E4F912
:1005CC00FA227818EF2FFFEE33FEED33FDEC33FCFF
:1005DC00C933C910D7059BE99A4007EC9BFCE99AF3
:1005EC00F90FD8E0E4C9FAE4CCFB2275F010EF2F38
:1005FC00FFEE33FEED33FDCC33CCC833C810D70738
:10060C009BEC9AE899400AED9BFDEC9AFCE899F872
:0E061C000FD5F0DAE4CDFBE4CCFAE4C8F92205
:0E062A00C3E49FFFE49EFEE49DFDE49CFC22E1
:10063800F8E0FBA3A3E0F925F0F0E582158270024B
:070648001583E0FA38F022EF
:09064F00EBF0A3EAF0A3E9F022AC
:10065800D083D082F8E4937012740193700DA3A331
:1006680093F8740193F5828883E473740293686045
:06067800EFA3A3A380DF45
:10200100EFC394304009EFC3943A5003D38001C326
:0120110022AC
:00000001FF
